:100000000C94C3020C94FB020C94FB020C94FB02B4
:100010000C94FB020C94FB020C94FB020C94FB026C
:100020000C94FB020C94FB020C942C260C94FE26E0
:100030000C940B210C94FB020C94FB020C94FB021D
:100040000C94FB020C94FB020C94FB020C94FB023C
:100050000C94FB020C9493210C94FB020C94FB0275
:100060000C94FB020C94FB020C94FB020C94FB021C
:100070000C94FB020C94FB020C94FB020C94FB020C
:100080000C94FB020C94FB020C94FB020C94FB02FC
:100090000C94FB020C94FB020C94FB020C94FB02EC
:1000A0000C94FB020C94FB020C94FB02CB05CB05D9
:1000B000F705F7055F067D06950795078806210772
:1000C000320732076B2792278A2892278A28DE2751
:1000D00001288A2858286728165C1F002100230061
:1000E000250027002E0049001E00200022002400C9
:1000F00026002D002A004B002B001A0015001C00C2
:100100000C00130030004C00140008001700180009
:1001100012002F0031004E003900160009000B00BC
:100120000E00330028000000040007000A000D0044
:100130000F00340000000000E1001B001900110056
:1001400036003800520051001D0006000500100066
:100150003700E50050004F00E000E300E2002C0013
:10016000E6000151E400000035003B003D003F0087
:10017000410043004500AE003A003C003E00400014
:100180004200440001004A000100C65CCA5C010054
:10019000010046004800A800C45CC85C01000100E2
:1001A0000100470001004D000100C75CCB5C01006D
:1001B0000100010001000000C35CC95C01000100F6
:1001C0000100010000000000010001000100010029
:1001D00001000100A900AA000100010001000100C6
:1001E00001000100AC00AB000100A75D0100005C54
:1001F000010001000100000000047F3F1F64321471
:10020000643214783C1E1E140A0522232526282950
:100210002A2C2D2F3032333536383A3B3D3E404282
:10022000434547494A4C4E5051535557595A5C5EC5
:100230006062646668696B6D6F71737577797B7DD9
:100240007F81838587898A8C8E90929496989A9CD8
:100250009E9FA1A3A5A7A8AAACAEAFB1B3B4B6B8F0
:10026000B9BBBCBEBFC1C2C3C5C6C7C9CACBCCCD52
:10027000CED0D1D2D2D3D4D5D6D7D7D8D9D9DADA2D
:10028000DBDBDBDCDCDCDCDCDDDDDDDDDCDCDCDCAD
:10029000DCDBDBDBDADAD9D9D8D7D7D6D5D4D3D2E1
:1002A000D2D1D0CECDCCCBCAC9C7C6C5C3C2C1BFBF
:1002B000BEBCBBB9B8B6B4B3B1AFAEACAAA8A7A523
:1002C000A3A19F9E9C9A98969492908E8C8A8987DF
:1002D0008583817F7D7B79777573716F6D6B6968BD
:1002E000666462605E5C5A5957555351504E4C4A91
:1002F0004947454342403E3D3B3A3836353332303C
:100300002F2D2C2A292826252322FFAA7F5540009D
:1003100001010101010101010102020202020202C6
:100320000202030303030303030304040404040499
:10033000040505050505060606060607070707075F
:1003400008080808090909090A0A0A0B0B0B0C0C12
:100350000C0D0D0D0E0E0E0F0F0F101011111112AE
:100360001213131414151516161717181819191A2D
:100370001A1B1B1C1D1D1E1E1F2020212222232490
:1003800024252626272829292A2B2C2D2D2E2F30CF
:10039000313232333435363738393A3B3C3D3E3FE3
:1003A000404142434445464748494A4C4D4E4F50D0
:1003B000515354555658595A5B5D5E5F616264658E
:1003C0006668696B6C6D6F7072737577787A7B7D18
:1003D0007E8082838587888A8C8E8F91939596986C
:1003E0009A9C9EA0A2A3A5A7A9ABADAFB1B3B5B788
:1003F000BABCBEC0C2C4C6C9CBCDCFD1D4D6D8DB5F
:10040000DDDFE2E4E7E9EBEEF0F3F5F8FAFDFF1EDD
:100410000342006C00610063006B0070006C0075AB
:10042000006D0020004B0065006500620000000EBA
:10043000035000690078006C007500700000000433
:1004400003090409023B00020100A0FA09040000AC
:1004500001030101000921110100012240000705EB
:1004600081030800010904010001030000000921C3
:100470001101000122B600070582032000011201CC
:100480000002000000085850504201100102000113
:1004900005010902A10185020901A100050919014F
:1004A000290815002501950875018102050109300B
:1004B00009311581257F9502750881060938158156
:1004C000257F950175088106050C0A3802158125DE
:1004D0007F950175088106C0C005010980A10185CD
:1004E0000319012AB700150126B70095017510817F
:1004F00000C0050C0901A101850419012AA00215FB
:100500000126A002950175108100C005010906A110
:10051000018506050719E029E715002501950875ED
:100520000181020507190029EF1500250195F075D5
:1005300001810205081901290595057501910295AA
:100540000175039101C005010906A101050719E024
:1005500029E71500250195087501810295017508A7
:1005600081010507190029FF150026FF0095067572
:100570000881000508190129059505750191029565
:100580000175039101C011241FBECFEFDAE0DEBF79
:10059000CDBF04B603FE18C080913403909135039B
:1005A000A0913603B09137038730904BA740B04BF2
:1005B00059F41092340310923503109236031092BE
:1005C0003703E0E0F8E3099511E0A0E0B1E0E6E4EC
:1005D000F3E502C005900D92A43CB107D9F723E0E2
:1005E000A4ECB1E001C01D92A433B207E1F70E9470
:1005F0007C130C94A1290C9400009C01FB018281C6
:10060000882381F0273A3D4571F48091DA0284FB1A
:10061000222720F991E0922790FB84F98093DA0257
:1006200080E0089581E0089581E008950C94FD0232
:1006300008950C9418031F93CF93DF9300D000D03C
:100640001F92CDB7DEB749835A836B833091C701C0
:1006500089819A81311114C0662359F0222349F00F
:100660000E94D209182F682F89819A810E947B09E4
:1006700003C00E94A609182F69817A81812F04C0C6
:100680000E94D20969817A810F900F900F900F908C
:100690000F90DF91CF911F910C94F710FC01262F42
:1006A000408151816281738184810C941B0381E0BC
:1006B0000895CF93DF93EC0160E00E944E03BE01EA
:1006C000DF91CF910C9419030C943C120C943812C6
:1006D00008950E9425080E9468032FEF84E39CE0A0
:1006E000215080409040E1F700C000000C94B921F7
:1006F0000F931F93CF93DF938C0161E00E944E0311
:10070000EC01B8010E941603882309F444C0B80123
:10071000CE010E94571F8823F1F1B801CE010E943B
:100720006B1D8823C1F1B801CE010E94B31E88233E
:1007300091F1B801CE010E94711C882361F1F8018A
:100740008281882309F1CB358DE5D807C1F050F4BB
:10075000C115FCE5DF0781F0CF3DDC45A9F40E941F
:10076000090F19C0CC35EDE5DE0761F0CD35DD456B
:1007700059F40E944C0E08C00E9469030CC00E94EC
:10078000550E02C00E94580EC801DF91CF911F91F3
:100790000F910C94140380E0DF91CF911F910F9182
:1007A00008950E94EE200E94EE030C94EE1A0E941F
:1007B000F1030E94BA1B0C94F42008950C94DD03FD
:1007C00081E008950C94E0030895CF93C82F0E9410
:1007D000DE038C2F0E94E203CF91089580E00C94F9
:1007E000E5030E94B31F0C94E5030E94B31F909190
:1007F000C601891721F08093C6010C94E503089582
:10080000CF93DF93CDB7DEB72B970FB6F894DEBF4B
:100810000FBECDBF4F83588769877A878B87611159
:100820000E94980D9E012F5F3F4F86E0F9011192C3
:100830008A95E9F785E0FE013796D90101900D927E
:100840008A95E1F789819A814C815D81452B31F050
:100850009F3F31F491E08F3F19F403C091E001C054
:1008600090E090FF09C049815A816B817C818D8124
:100870009E810E94B90C05C0C9010E9457038111D5
:10088000F2CF2B960FB6F894DEBF0FBECDBFDF912F
:10089000CF910895FC01808191810E94140A0895EE
:1008A000CF93882309F4A4C0C82F8238C1F40E94D2
:1008B000B31F81FD9DC069E3809102019091030106
:1008C0000E94A9200E94BA0D2FEF81EE94E02150E2
:1008D00080409040E1F700C0000069E319C0833810
:1008E00001F50E94B31F80FD83C063E58091020182
:1008F000909103010E94A9200E94BA0D2FEF81EE72
:1009000094E0215080409040E1F700C0000063E592
:1009100080910201909103010E94B420CF910C9428
:10092000BA0D8438C1F40E94B31F82FD61C067E430
:1009300080910201909103010E94A9200E94BA0DAA
:100940002FEF81EE94E0215080409040E1F700C00D
:10095000000067E4DDCF8CEF8C0F813AD0F46C2F70
:1009600080910201909103010E942920882349F07F
:100970006C2F80910201909103010E94B4200E948B
:10098000BA0D6C2F80910201909103010E94A92061
:10099000C5CF80E28C0F883048F4C77081E001C079
:1009A000880FCA95EAF70E947B0DB8CFEBE5EC0FF4
:1009B000E33040F4F0E0E65AFE4F808190E0CF91C2
:1009C0000C94E71FE8E5EC0FE73150F4F0E0EE0F90
:1009D000FF1FE45DFE4F80819181CF910C94FD1F3C
:1009E000CD3E30F08C2F0E940114CF910C94D31483
:1009F000CF910895882309F464C0823879F40E9465
:100A0000B31F81FF5EC069E38091020190910301F1
:100A10000E94A9200E94BA0D69E310C08338B1F486
:100A20000E94B31F80FF4DC063E580910201909149
:100A300003010E94A9200E94BA0D63E58091020182
:100A4000909103010E94B4200C94BA0D843879F47B
:100A50000E94B31F82FF35C067E48091020190912C
:100A600003010E94A9200E94BA0D67E4E7CF9CEF22
:100A7000980F913A10F4682FE1CF90E2980F9830D8
:100A800050F4877091E001C0990F8A95EAF7892F99
:100A90000E94810DD9CF9BE5980F933020F480E020
:100AA00090E00C94E71F98E5980F973120F480E0D0
:100AB00090E00C94FD1F8D3E20F00E945C140C947D
:100AC000D31408951F93CF93DF93182FEB010E9447
:100AD0005004209741F08FE99FE00197F1F700C0A3
:100AE00000002197F6CF812FDF91CF911F910C94B9
:100AF000FA04893319F060E070E002C060E570E04C
:100B00000C946205882321F00E947B0D0C94BA0D91
:100B10000895882321F00E94810D0C94BA0D089548
:100B2000CF92DF92EF92FF920F931F93CF93DF93B9
:100B30007C01D62FC72FFC011281058102950F7011
:100B40000E94710D8823B9F01123A9F08C2F807FAA
:100B5000803421F080E28D0F883068F08091DB02D4
:100B600082FD09C082E00E941A0E0E94710D91E080
:100B7000D82ED92601C0D12CCC2EC2948FE0C82209
:100B80008C2D90E08C30910508F0CFC1FC01EA5A21
:100B9000FF4F0C9408298C2F807FCF70882311F091
:100BA000C295C07F112399F0CC2309F4AAC180E239
:100BB0008D0F883010F0D11104C08C2F0E947B0D56
:100BC00003C08C2F0E948B0D0E94BA0D9AC18D2FED
:100BD0000E94FA04CC2309F4A8C180E28D0F88306A
:100BE00038F1DD2329F18C2F0E94910D24C08C2F28
:100BF000807FCF70803211F0C295C07FDD2319F065
:100C0000D130A1F13DC08091DB0282FF17C01123DA
:100C100049F0CC2329F08C2F0E947B0D0E94BA0D45
:100C200080E070C180E00E94FA04CC2309F47DC109
:100C30008C2F0E94810D0E94BA0D77C1112371F093
:100C4000002341F0013031F40E949B0D8C2B0E9457
:100C5000A30D6BC10E949B0D8C2B1DC0002319F0AE
:100C6000013009F462C10E94B00D25C0112321F0AA
:100C7000063008F05AC10EC0053008F056C11BC03E
:100C8000112361F0002331F0F701858180FF39C124
:100C90008F7085838C2F0E94820547C1002359F0F5
:100CA000D93309F03FC1FFEF07EE13E0F1500040E8
:100CB0001040E1F735C18C2F0E94890536C18C2F79
:100CC00086958695837019F0813061F02EC11123CD
:100CD00021F08D2F9C2F937002C080E090E00E9445
:100CE000E71F2BC1112321F08D2F9C2F937002C081
:100CF00080E090E00E94FD1F20C18D2F112319F08C
:100D00000E94011402C00E945C140E94D31415C1F9
:100D10008C2F837009F047C011110BC12D2F229524
:100D200026952770220F220F6D2F6F70862F90E06F
:100D3000A0E0B0E0022E04C0880F991FAA1FBB1FBD
:100D40000A94D2F7D4FF10C04FE050E060E070E0AA
:100D500004C0440F551F661F771F2A95D2F7409590
:100D600050956095709503C040E050E0BA01C6957B
:100D7000C695C3708A019B01082B192B2A2B3B2B8C
:100D8000C901B801C23049F058F4C13019F00E94CD
:100D90009108CFC00E947F08CCC00E94A308C9C0A0
:100DA0000E947D08C6C0112319F08C2F817001C0EC
:100DB0008695882309F4BDC02D2F2295269527708E
:100DC000220F220F6D2F6F70862F90E0A0E0B0E011
:100DD000022E04C0880F991FAA1FBB1F0A94D2F7C6
:100DE000D4FF10C04FE050E060E070E004C0440F5A
:100DF000551F661F771F2A95D2F74095509560952D
:100E0000709503C040E050E0BA01C695C695C37026
:100E10008A019B01082B192B2A2B3B2BC901B801F6
:100E2000C23049F058F4C13019F00E94560981C00F
:100E30000E9444097EC00E9468097BC00E94B708D6
:100E400078C0CF70112339F08C2F0E94DD088D2FD0
:100E50000E9482056EC08D2F0E9489058C2F0E94F2
:100E6000FE0867C0D23F21F128F4D03F41F0D13FC6
:100E7000C1F043C0D33F19F1D43F79F03EC01123F4
:100E800041F0053008F051C08C2F8F710E9423096A
:100E90004CC0063008F049C0F7CF8091DB0282FFDA
:100EA00018C0112339F08C2F8F710E94DD083DC0CE
:100EB0001123C9F38C2F8F710E94FE0836C01123B5
:100EC00029F08C2F8F710E94C8082FC00E94C30880
:100ED0002CC0112349F0CF718C2F0E94DD0863E0F4
:100EE0008C2F0E94FF0D21C081E00E941A0E02305B
:100EF000E0F082E00E941A0E18C0112331F00023A6
:100F000091F28D2F0E94500410C0002399F2D93322
:100F100049F41FEF27EE33E0115020403040E1F755
:100F200000C000008D2F0E94FA0488EF8C0D8430E1
:100F300020F40E94B31F0E94E503DD20C9F00E9447
:100F40006D0D80FD15C0F70112820E94670D0E9491
:100F5000DD08C7010E94D9070E94670DDF91CF917C
:100F60001F910F91FF90EF90DF90CF900C94FE08AF
:100F7000DF91CF911F910F91FF90EF90DF90CF9075
:100F800008950F931F93CF93DF93EC0168817981CC
:100F90008A810E941F0A8C010E947A090E946B08B4
:100FA000B801CE010E949005DF91CF911F910F9162
:100FB0000895CF93DF93EC01988189812B813C8147
:100FC000232B31F08F3F31F481E09F3F19F403C0B0
:100FD00081E001C080E080FD1DC0CE010E94780349
:100FE000811110C00E94710D8823A1F08A8188238D
:100FF00089F08091DB0282FD0DC082E0DF91CF910C
:101000000C941A0ECE010E94C107CE01DF91CF9140
:101010000C945903DF91CF91089580E090E00E94F5
:10102000E71F80E090E00E94FD1F0E94980D0E9443
:10103000BA0D0E9404160C94D31480910201909171
:1010400003010E94BF200C940D080E94880D0C948F
:101050001D0892959F70963079F010F4925001C05F
:101060009A50923068F4803F69F018F4883E40F45A
:1010700009C0843F29F406C0883E20F0813F11F06A
:1010800080E0089581E00895FC01808191810E94B3
:10109000140A0E9429080895CF93DF9300D000D04E
:1010A0001F92CDB7DEB70F900F900F900F900F905B
:1010B000DF91CF910895CF93DF9300D000D000D07F
:1010C000CDB7DEB726960FB6F894DEBF0FBECDBF04
:1010D000DF91CF910895089508950C946C080C94B5
:1010E0006D080E946F086093F9017093FA01809374
:1010F000FB019093FC010C940D080C9471080F9364
:101100001F930091F9011091FA012091FB01309198
:10111000FC01602B712B822B932B1F910F910C9450
:1011200071080F931F930091F9011091FA0120911A
:10113000FB013091FC0160237123822393231F91D3
:101140000F910C9471080F931F930091F901109166
:10115000FA012091FB013091FC0160277127822761
:1011600093271F910F910C9471080C946C080E94A6
:10117000B5086093F5017093F6018093F7019093A1
:10118000F8010C940D0860E070E0CB010C94B708F6
:101190000F931F9341E050E060E070E08A019B01F3
:1011A00004C0000F111F221F331F8A95D2F7C901F7
:1011B000B8011F910F910C94B7080F931F9341E052
:1011C00050E060E070E004C0440F551F661F771FB9
:1011D0008A95D2F78091F5019091F601A091F701DF
:1011E000B091F8018A019B01082B192B2A2B3B2B6C
:1011F000C901B8011F910F910C94B7080F931F9369
:1012000041E050E060E070E004C0440F551F661FED
:10121000771F8A95D2F7409550956095709580918B
:10122000F5019091F601A091F701B091F8018A01C2
:101230009B01082319232A233B23C901B8011F91CD
:101240000F910C94B7080F931F9341E050E060E0BA
:1012500070E004C0440F551F661F771F8A95D2F7B0
:101260008091F5019091F601A091F701B091F801FC
:101270008A019B01082719272A273B27C901B801A2
:101280001F910F910C94B7080F931F930091F501D4
:101290001091F6012091F7013091F801602B712B2C
:1012A000822B932B1F910F910C94B7080F931F93D0
:1012B0000091F5011091F6012091F7013091F801AC
:1012C00060237123822393231F910F910C94B708FD
:1012D0000F931F930091F5011091F6012091F701F2
:1012E0003091F80160277127822793271F910F9172
:1012F0000C94B708089528E0929F800D1124E82FE0
:10130000E695E695E695877051E001C0550F8A9500
:10131000EAF785E0E89FF0011124E853FE4F20E052
:1013200030E070E04081CB01022E02C09695879597
:101330000A94E2F78170819584278523842781931D
:101340002F5F3F4F2530310569F7089528E0929FC0
:10135000800D1124682F669566956695982F977075
:1013600085E0689FB001112440E050E080E0FB017F
:10137000E40FF51FE853FE4F208130E0092E02C034
:10138000369527950A94E2F721703327042E01C081
:10139000220F0A94EAF7822B4F5F5F4F45305105C9
:1013A00031F70895BF92CF92DF92EF92FF920F93A1
:1013B0001F93CF93DF938C01C090F501D090F6017D
:1013C000E090F701F090F8018091F9019091FA0115
:1013D000A091FB01B091FC01C82AD92AEA2AFB2A74
:1013E000CFE1D0E0D701C6010C2E04C0B695A79579
:1013F000979587950A94D2F780FD04C0219790F7BE
:10140000B12C07C0BC2EB8018C2F0E940C11019783
:10141000A9F38B2DDF91CF911F910F91FF90EF904A
:10142000DF90CF90BF900895CF93DF93EC010E949F
:10143000D209BE010E940C11DF91CF9108951F9334
:10144000CF93DF93EB019091C701992321F0CB015A
:101450000E94140A13C0882349F0CB010E94D209CC
:10146000182F682FCE010E947B0904C0CB010E9477
:10147000A609182FBE01812F0E940C11DF91CF9178
:101480001F9108951F93CF93DF93C091FD0116E044
:101490008091FE01C81799F0D0E01C9FF0011D9FBC
:1014A000F00D1124E150FE4F408151816281738122
:1014B000848195810E945B082196C770E9CFDF91F6
:1014C000CF911F91089540912F0250913002609169
:1014D00031027091320280913302909134020C9467
:1014E0005B08EF92FF920F931F93CF93DF9380914E
:1014F000340282958F7009F065C080913102882393
:1015000009F460C08091FD01F090FE0110912F025E
:1015100000913002609132027091330291E01F3FDE
:1015200009F090E0C0910001D0910101292F96E0CF
:10153000E92E8F1509F446C06115710521F00F3FA2
:1015400021F030E003C031E001C0322F90E030FDE7
:1015500036C0E89EF001E99EF00D1124DF01A15094
:10156000BE4F11963C911197301329C03C91311315
:1015700026C012963C911297311121C013964D91BD
:101580005C911497461B570B4C175D07C0F4809174
:1015900034028F70806180933402EC5FFD4F808154
:1015A0008F70806180838FE292E00E94D907DF9183
:1015B000CF911F910F91FF90EF900C94420A0196EA
:1015C0008770B7CFDF91CF911F910F91FF90EF9070
:1015D00008959F92AF92BF92CF92DF92EF92FF92C7
:1015E0000F931F93CF93DF93CDB7DEB761970FB6FD
:1015F000F894DEBF0FBECDBF8C0185E0F801DE019F
:101600001D9601900D928A95E1F7D8011296EC9003
:1016100090912F02E09130022091320230913302FA
:101620002115310531F0EF3F31F481E09F3F19F48E
:1016300003C081E001C080E0B82FB1709B2E80FD17
:1016400047C1D8014C9111965C9111971396AD90BA
:10165000BC9014978FE2C82E82E0D82EF090310211
:10166000B501621B730B2091000130910101FF2035
:1016700009F4D9C0809134026217730708F095C04D
:10168000282F207F09F052C05E1313C0491311C0E8
:10169000FE2CE1100EC08F708061809334020E9496
:1016A000630AC6010E94D90780913402F80185833C
:1016B0004DC1AB2831F05F3F31F481E04F3F19F469
:1016C00003C081E001C080E080FD03C081E08E2581
:1016D00002C080E090E0F82FF170FF2E80FF1CC068
:1016E0008091FD012091FE0136E0821709F40BC1C3
:1016F00090E0389FF001399FF00D1124E150FE4F2A
:101700006181561306C06081461303C06281E612F0
:1017100003C001968770E9CFFE2CEE2009F416C1B4
:101720008091340281608093340254C05E1306C0FD
:10173000491304C0E11002C0F80199C0C8010E9419
:101740004408882361F1EE2051F120913402822F68
:1017500082958F7090E0029774F080912F029091A3
:10176000300298878F831986BB86AA862C87CE0184
:1017700007960E94D90786E0F801AFE2B2E0019037
:101780000D928A95E1F70E94710A0E94630A0AC0CD
:101790005E1711F1C8010E94440881112CC0C801D4
:1017A0000E94D907FF24F394D1C0282F207F81F70E
:1017B0007A2DB98AA88A6E2D89890E944C088FE2F9
:1017C00092E00E94D90786E0D6011D928A95E9F73A
:1017D0000E94630AF12CBAC04913DCCFE110DACFC2
:1017E000F8018583C8010E94D90786E0D6011D92C1
:1017F0008A95E9F7ABC0EE2091F220913402822F56
:1018000082958F7090E002970CF4B5CF80912F02F3
:10181000909130029A8389831B82BD82AC822E8391
:10182000CE010196A6CF6217730708F044C0FE2CC4
:10183000EE2009F4B4CF5E1330C049132EC02091BE
:10184000340220FD21C0822F82958F70482F50E0F6
:1018500041155105C9F0F80125834F30510541F07C
:101860008F5F982F9295907F822F8F70892B858321
:10187000C8010E94D90786E0F801AFE2B2E001900A
:101880000D928A95E1F73CC086E0F801AFE2B2E044
:1018900001900D928A95E1F759C0C8010E94440851
:1018A000811169CF80913402816080933402C80134
:1018B0000E94D9074BC07A2DB98AA88A6E2D8989D2
:1018C0000E944C0886E0D6011D928A95E9F718C05F
:1018D000EE2009F464CFC8010E944408F82E882342
:1018E00009F45DCF86E0F801AFE2B2E001900D921D
:1018F0008A95E1F78FE292E00E944A040E94710A01
:101900000E94630A23C04D875E878D859E850E9455
:10191000140A292F22952F70223028F49F7039F055
:10192000811105C00BC0243028F49F7049F4805EFB
:10193000883020F0C8010E94D9079F2CF92C06C0DE
:10194000D80115969C91907F91F7F8CF8F2D6196D5
:101950000FB6F894DEBF0FBECDBFDF91CF911F91C0
:101960000F91FF90EF90DF90CF90BF90AF909F903E
:1019700008951F93CF93DF93CDB7DEB72C970FB6A3
:10198000F894DEBF0FBECDBF4F83588769877A8733
:101990008B879C87CE0107960E94E90A8823D1F0A5
:1019A0009F8188852A853B85232B31F08F3F31F439
:1019B00081E09F3F19F403C081E001C080E080FD19
:1019C00047C04F81588569857A858B859C850E94A3
:1019D0005B083EC086E0FE013796DE01119601905D
:1019E0000D928A95E1F7FF81E8856A857B8561150F
:1019F000710531F0EF3F31F481E0FF3F19F403C08E
:101A000081E001C080E080FD23C02091FE0130E034
:101A1000C9010196877099274091FD0150E0841714
:101A20009507F1F1F983EA837D836C8396E0929FB9
:101A3000D001939FB00D1124A150BE4FFE013196ED
:101A400001900D929A95E1F78093FE010E94420A5F
:101A500016E08091FD019091FE01891771F1189FA8
:101A6000C001112481509E4F0E94E90A882329F168
:101A7000E091FD011E9FF0011124E150FE4F4081D5
:101A8000518162817381848195810E945B0880917C
:101A9000FD0190E00196877099278093FD01D9CFD1
:101AA0000E9425081092FE011092FD01EFE2F2E083
:101AB00086E0DF011D928A95E9F72C960FB6F8941F
:101AC000DEBF0FBECDBFDF91CF911F9108958091F2
:101AD0005502859585958595089580915502877065
:101AE000089590915502977081E009F480E008957F
:101AF00080917802089590917802892B80937802E2
:101B000008958095909178028923809378020895B2
:101B100010927802089590917702892B8093770232
:101B20000895809590917702892380937702089594
:101B300010927702089580915602089508950C94AA
:101B40009E0D0C949F0D9091DB0292FD08C0909128
:101B50005602981721F0809356020C94A10D089517
:101B600080915602882329F01092560280E00C944E
:101B7000A10D0895CF93DF93E0910201F09103014D
:101B8000809178028083E0910201F09103019081BD
:101B900080917702892B808380915602882381F07F
:101BA000E0910201F09103019081892B8083809163
:101BB0000201909103010E94132081110E94B00D37
:101BC000C0910201D091030140E250E065E372E070
:101BD000CE010E944C29892B69F080E2FE01A5E329
:101BE000B2E001900D928A95E1F7CE01DF91CF919D
:101BF0000C94BF1FDF91CF9108950C949E0D90918E
:101C0000DB0292FD10C098E0899F90011124262BE1
:101C1000209355020E94DD08809155028595859597
:101C200085950C94FD0D0C94DD081092550280E012
:101C30000C94FD0D209155028095822380935502CE
:101C4000982F977099F430E0482F082E000C550B10
:101C50002417350759F09091DB0292FD07C0859556
:101C6000859585950E94FE080C94150E0895909117
:101C7000DB0292FB222720F9281769F080FB92F9FA
:101C80009093DB028091DA029091DB020E94850E34
:101C900082E00C941A0E08958091DB0282FB882763
:101CA00080F991E089270C94370E81E00C94370E6F
:101CB00080E00C94370E6FEF7FEF80E090E00C94A3
:101CC0008B2980E090E00E94672921E0893E9E4FA9
:101CD00009F020E0822F089582E090E00C945929C9
:101CE00083E090E00C945929CF9384E090E00E9427
:101CF0005929C82F82E290E00E9459292C2F30E008
:101D0000A901582BCA01CF910895CF93C92F682FED
:101D100084E090E00E946D296C2F82E290E0CF91E8
:101D20000C946D29AB01BC018FE090E00C947F29ED
:101D3000AB01BC0183E190E00C947F2960E070E08E
:101D4000CB010C94980E60E070E0CB010E94920EE3
:101D50000C949E0E69EE7EEF80E090E00E948B294D
:101D600060E082E090E00E946D2960E083E090E016
:101D70000E946D291092F9011092FA011092FB0154
:101D80001092FC0160E084E090E00E946D2960E028
:101D900082E290E00E946D2960E085E090E00E9480
:101DA0006D2960E086E090E00E946D296FEF87E08A
:101DB00090E00E946D2940E050E0BA0188E090E098
:101DC0000E947F2960E08DE090E00E946D2940E054
:101DD00050E0BA0188E190E00E947F2960E087E14D
:101DE00090E00E946D2940E050E0BA018CE190E063
:101DF0000E947F2960E070E080E290E00E948B29E1
:101E000040E050E0BA0188E190E00E947F290C9404
:101E1000A30E0C94AA0E682F8EE090E00C946D290E
:101E20000E947821609386027093870280938802D3
:101E3000909389026093820270938302809384025C
:101E400090938502089585B7806885BF85B78068BF
:101E500085BF089581E008950C942A0F08950C948D
:101E60002E0F0C942E0F0C94310F0C942E0F0C94FB
:101E7000350F0C942E0F0E94230F88EE91E10E94E3
:101E8000A91F0E94390F0C94370F0E942F0F0C943A
:101E90002E0F0E9402120C94E4030E9463210E9400
:101EA000D9120E94490F0E947F1B0C94330F8F920E
:101EB0009F92AF92BF92CF92DF92EF92FF920F93D9
:101EC0001F93CF93DF93CDB7DEB72A970FB6F89461
:101ED000DEBF0FBECDBF0E94EE12982E81110E9470
:101EE000100F89E7A82E82E0B82E00E010E0802EC7
:101EF000802F0E942612D82EF501C1905F01C826BE
:101F0000B1F40F5F1F4F0930110589F78FEF8983F7
:101F10008A831B820E946C218160782F9D838C8331
:101F200049815A816B818D810E9400042FC080916C
:101F30008A0281FD0E942C12E12CFF24F3948C2D47
:101F40008F21F1F00E942C0F882399F0EE828F826E
:101F5000DF2081E009F480E088870E946C218160A5
:101F6000782F9A8789874E815F8168858A850E944C
:101F70000004F801E758FD4F8081F826F08206C082
:101F8000E394FF0CF8E0EF12DACFBBCF81E09110C1
:101F900001C080E02A960FB6F894DEBF0FBECDBF19
:101FA000DF91CF911F910F91FF90EF90DF90CF9035
:101FB000BF90AF909F908F9008950E94570F0E94FE
:101FC000C31B0E94F1140C94F503CF93DF930E947E
:101FD0001111EC01811521E5920708F045C081152A
:101FE00030E5930708F094C0883E910528F5803EBF
:101FF000910508F0F8C0883A910570F4853A91058A
:1020000008F07CC08130910509F475C008F4E8C07F
:10201000049708F0E8C0E4C08F3B910508F0E0C0E9
:10202000C85AD0E0CC0FDD1FC35ADE4F0990D881CB
:10203000C02DCE019464D8C0811540E2940758F4B5
:10204000811551E0950708F0CEC08D3E910508F44A
:10205000C7C09065C9C0C11580E4D80708F4C0C0E6
:10206000DF70CE01906AC0C0811525E59207A8F403
:10207000811534E5930708F095C0811543E5940771
:1020800008F07BC0811552E5950708F061C0D82F94
:10209000CC27CE01816F906AA7C0C11589E5D8070A
:1020A000A0F4C11528E5D20708F082C0C11536E5B5
:1020B000D30708F095C08C2F0E94A5118F7190E076
:1020C000D82FCC27CE0190628FC0C1154AE5D40726
:1020D00008F474C0CE0190568115904208F080C07B
:1020E0008D2F8F710E94A511DD27D0628F71AE01F7
:1020F000582BCA0179C081E090E076C0C55AD0E083
:10210000C557DE4F8881C82FD0E0CE0190646CC0E7
:1021100074E0969587957A95E1F7282F23703C2FE8
:10212000337081E090E002C0880F991F3A95E2F782
:102130009C68AC01522B9A019C2F9F7096959695A6
:1021400050E2959FE0011124C9018C2B9D2B4CC0BE
:102150008370992721E030E002C0220F331F8A9557
:10216000E2F79C2F9695969580E2989FE0011124C6
:10217000C22BD32BCE019C6837C08370992721E0F6
:1021800030E002C0220F331F8A95E2F79C2F96950C
:10219000969540E2949FE0011124C22BD32BCE01EF
:1021A0009A6822C0D82FCC27CE01846F906A1CC0B9
:1021B000DC2FCC27CE01806F906A16C08C2F8F70D9
:1021C0000E94A51194E0D695C7959A95E1F7CF7036
:1021D000D0E0DC2FCC27D0699E01282BC90104C098
:1021E00080E090E001C0CE01DF91CF910895E72F0C
:1021F000F0E099E0899FE00DF11D112483E0EE0FDE
:10220000FF1F8A95E1F7E60FF11DEE0FFF1FE85261
:10221000FF4F8591949108950E94F7100E94E50F59
:1022200008958238910569F1B0F48133910509F47C
:102230006DC048F48932910509F463C08A32910572
:1022400009F469C008958533910509F455C08933AF
:102250009105B9F00895833E910569F138F4803E07
:102260009105B1F0823E910509F10895863E9105F0
:10227000A9F1873E9105B9F1843E910509F064C04A
:1022800023C02091DA0220FD4FC021FD4DC00895EA
:102290008091DA0280FD44C08091DB0280FF44C05F
:1022A0008091DA0284FD42C083EE4DC08091DA0253
:1022B00082FF38C0F5CF8091DA0282FD33C0809171
:1022C000DB0280FD31C0ECCF8091DB0281FF32C0A8
:1022D0008091DA0284FD2AC087EE35C08091DA024F
:1022E00083FF26C0F5CF8091DA0283FD21C0809163
:1022F000DB0281FD1FC0ECCF8091DA0285FD1CC09E
:102300001DC08091DA0285FD19C016C08091DA02E5
:1023100086FD16C017C08091DA0286FD13C010C07A
:1023200089E311C082EE0FC080EE0DC080E00BC0CB
:1023300086EE09C084EE07C089E205C085E303C0CC
:102340008AE201C081E390E008959091DA0292FF61
:102350000DC0282F2871283019F4877F846006C0AB
:10236000282F2471243011F48B7F886093FF0DC0D7
:10237000282F2871283119F4877E846106C0282F00
:102380002471243111F48B7E88612091DB0220FFBF
:102390000DC0382F3871383019F4877F816006C03E
:1023A000382F3171313011F48E7F886021FF0DC0DC
:1023B000282F2871283119F4877E816106C0282FC3
:1023C0002171213111F48E7E886194FD877E0895FC
:1023D00080E008950C945B0E0E94EE128FE39CE95E
:1023E0000197F1F700C000000E94EE1280E00E9409
:1023F000261280FF04C00E94EA110C94B9210895AE
:102400000C94EC110E94610E811102C00E94090F10
:102410000E946C0E80938A020E94740E9093DB02DD
:102420008093DA020E9400120E94700E682F70E002
:1024300080E090E00E947D086091F5017091F601C6
:102440008091F7019091F8010C94B508E82FF0E025
:10245000EB51FD4F80810895089580EA8A95F1F748
:10246000089500C008950C942D1208950C9435120F
:102470000C9436120C9435120C943A12F894E82FFE
:10248000E295EF70F0E031A1282F2F7081E090E00D
:1024900001C0880F2A95EAF7982F9095932391A36E
:1024A00092A1892B82A3789408950F931F93CF93C1
:1024B000DF93C6E9D1E089918F3F11F00E943E126F
:1024C00081E0CF39D807B9F7CEE8D1E006E911E0CD
:1024D00089918F3F11F00E943E120C171D07C1F722
:1024E000DF91CF911F910F910895CF92DF92EF92DC
:1024F000FF920F931F93CF93DF938C01C62FD0E0F1
:10250000CE018A569E4F7C01FC0190819F3F09F4C9
:1025100047C0D62EF894E92FE295EF70F0E081A144
:102520009F7021E030E001C0220F9A95EAF7822BDC
:1025300081A382A12095282322A378940E9431129E
:10254000EEE8F1E046E951E031E0C12C21912F3F66
:1025500089F0A22FA295AF70B0E090968C9190E098
:102560002F7002C0959587952A95E2F780FD02C0ED
:10257000832F01C080E0C82A330F4E175F0731F761
:10258000F70180818F3F11F00E943E1261E0C1107F
:1025900001C060E08D2D0E943312C00FD11FC88290
:1025A000DF91CF911F910F91FF90EF90DF90CF902F
:1025B00008950E94551289E0E5EEF2E0DF01982FC0
:1025C0001D929A95E9F7ECEDF2E0DF011D928A95F4
:1025D000E9F789E00E9439130C946403FF920F938A
:1025E0001F93CF93DF93CDB7DEB729970FB6F8943B
:1025F000DEBF0FBECDBF8E010F5F1F4F89E0F80118
:1026000011928A95E9F7F12C6F2DC8010E9475127D
:10261000F394F9E0FF12F8CF49E050E0B8018CEDF7
:1026200092E00E944C29FF24F394009709F4F12CC6
:10263000892B41F089E0F801ACEDB2E001900D92F8
:102640008A95E1F72F2D49E065EE72E08CED92E07E
:102650000E943A130E9466038F2D29960FB6F894B4
:10266000DEBF0FBECDBFDF91CF911F910F91FF90C5
:1026700008950895FF920F931F93CF93DF938C01DA
:10268000F62ED72FC42F222349F081E080938D02AC
:102690000E946C2190938C0280938B0280918D021A
:1026A0008823C1F080918B0290918C020E9484213A
:1026B000059780F0EF2DFD2FD8014C2F50E0CD0174
:1026C000801B910B841795071CF48D918193F7CF94
:1026D00010928D02DF91CF911F910F91FF9008957D
:1026E0000E9484230E944D0F0C9490230E949423F7
:1026F0000E94DD0F0C94AE230E940A210E946B23DE
:102700000E943B0F0E9470130E9476130E94450F97
:10271000FBCF8091940280FF06C06091090170E0B8
:10272000660F771F26C081FF04C06091090184E015
:1027300005C082FF07C06091090188E0689FB00171
:10274000112417C0909193029923D1F06091080150
:10275000961788F72091090188E0289F900111249D
:10276000929FA001939F500D112470E0CA010E9416
:10277000D2286038710540F46115710519F406C05E
:1027800068E070E0862F08958FE7089581E008954E
:102790008091940280FF08C06091050170E07595FA
:1027A00067957595679521C081FF06C06091050109
:1027B00070E07595679519C082FF04C060910501AE
:1027C00070E010C090919202992399F060910401F9
:1027D0009617A0F780910501899FC001112470E030
:1027E0000E94D2286038710540F46115710519F412
:1027F00006C061E070E0862F08958FE7089581E0BC
:1028000008958D3E21F40E948913819504C08E3E67
:1028100029F40E9489138093980208958F3E21F431
:102820000E948913819504C0803F29F40E94891376
:10283000809397020895893F19F40E94C81305C038
:102840008A3F31F40E94C8138195809399020895BC
:102850008B3F21F40E94C813819504C08C3F29F45A
:102860000E94C81380939A0208959FE0980F9830B1
:1028700078F421E030E0A90102C0440F551F9A9579
:10288000E2F7CA0190919602892B809396020895EF
:102890008D3F21F48091940281600BC08E3F21F422
:1028A00080919402826005C08F3F29F48091940248
:1028B00084608093940208958D3E39F4909198023B
:1028C00097FF35C01092980259C08E3E29F490911E
:1028D00098021916BCF32BC0909197028F3E29F4F1
:1028E00097FF25C01092970249C0803F19F419162E
:1028F000CCF31DC090919902893F29F41916BCF4BC
:10290000109299023BC08A3F19F497FF10C0F8CF8C
:102910008B3F39F490919A0297FF09C010929A0266
:102920002DC08C3F21F490919A021916BCF39FE0C0
:10293000980F983080F421E030E0A90102C0440FE4
:10294000551F9A95E2F7CA018095909196028923C6
:102950008093960213C08D3F21F4809194028E7F64
:102960000BC08E3F21F4809194028D7F05C08F3F74
:1029700029F4809194028B7F809394028091970236
:10298000811106C080919802811102C010929302B9
:1029900080919902811106C080919A02811102C032
:1029A0001092920208950E946C21209197022111A9
:1029B00004C020919802222321F0909391028093E9
:1029C000900220919902211104C020919A022223A1
:1029D00021F090938F0280938E0285E992E00C940F
:1029E000D91FEF92FF920F931F93CF93DF9300D0E5
:1029F00000D000D0CDB7DEB786E0E5E9F2E0DE0139
:102A0000119601900D928A95E1F7E0909702F0906F
:102A100098020091990210919A02109297021092D6
:102A200098021092990210929A02E11003C0FF20BE
:102A300009F45DC080919002909191020E948421DE
:102A4000AC0190919302992339F020910A0130E072
:102A50002417350758F04BC020910B018AE0289FBE
:102A6000900111242417350718F041C09F3F19F039
:102A70009F5F90939302EE2061F00E9489131E14D1
:102A800014F09FEF01C091E0989F902D1124909336
:102A90009702FF2061F00E9489131F1414F09FEF2A
:102AA00001C091E0989F902D11249093980230914D
:102AB00097023323E1F0209198022223C1F045EBE5
:102AC0003403C0011124992319F09093970203C095
:102AD00081E08093970235EB2303C00111249923F1
:102AE00019F09093980203C081E08093980201113D
:102AF00003C0112309F45DC080918E0290918F0272
:102B00000E948421AC0190919202992339F0209186
:102B1000060130E02417350758F04BC0209107011B
:102B20008AE0289F900111242417350718F041C02E
:102B30009F3F19F09F5F90939202002361F00E94E3
:102B4000C813101614F09FEF01C091E0989F902DCC
:102B5000112490939902112361F00E94C813111659
:102B600014F09FEF01C091E0989F902D1124909355
:102B70009A02309199023323E1F020919A022223A4
:102B8000C1F045EB3403C0011124992319F090934F
:102B9000990203C081E08093990235EB2303C001C1
:102BA0001124992319F090939A0203C081E0809335
:102BB0009A028091970281110BC080919802811135
:102BC00007C080919902811103C080919A028111FE
:102BD0000E94D314EB82FC820D831E8386E0FE01EB
:102BE0003196A5E9B2E001900D928A95E1F726961B
:102BF0000FB6F894DEBF0FBECDBFDF91CF911F910E
:102C00000F91FF90EF900895E5E9F2E086E0DF0193
:102C10001D928A95E9F710929302109292021092F7
:102C200094020895EF92FF920F931F93CF93DF9337
:102C30008B01682F11110AC0442329F0E82FF0E01E
:102C4000E15FFC4F6491762F862F75C0212F30E015
:102C5000E82FF0E0442321F0E15FFC4FE491F0E045
:102C600046E0049FC0011124CFEFD0E0BE010E94D6
:102C7000BE284BEA4603C001479F900D1124800FE8
:102C8000911D800F911D982F990F890FAE01421B46
:102C9000530B4E9FD0014F9FB00D5E9FB00D11247E
:102CA0009B2F189FA0011124452F55278E01041B2F
:102CB000150B0E9FA0010F9F500D1E9F500D11244C
:102CC0007E01E81AF108E29E8001E39E100DF29E5B
:102CD000100D1124212F3327C21BD30BCE9F90013F
:102CE000CF9F300DDE9F300D112462307105A9F0A9
:102CF00048F46115710569F061307105C9F48B2FD5
:102D0000752F0DC06430710581F058F06630710583
:102D100079F47E2F8B2F932F0DC0832F7B2F9E2F27
:102D200009C08E2F7B2F952F05C08E2F732F02C0C9
:102D30007E2F852F692FDF91CF911F910F91FF90EB
:102D4000EF90089541E00E941216089508950E94A0
:102D5000A2160895CF93DF93762FE901682F842F71
:102D60000E94A716798368838A83DF91CF910895A3
:102D70008091EE02282F269530E02115310519F4B7
:102D80008170826005C02532310524F0817088642D
:102D90008093EE02089588E090E00C946129CF9230
:102DA000DF92EF92FF926B017C010E94B816B7018F
:102DB000A60188E090E0FF90EF90DF90CF900C9418
:102DC0007F29EEEEF2E083E0808311828FEF828331
:102DD0008383148260817181828193810C94CF16E8
:102DE0008091EE0280FF02C08695089580E00895EC
:102DF0009091F202933018F49F5F9093F20288232F
:102E000051F06091EE027091EF028091F00290918A
:102E1000F1020C94CF16089581E00C94F81690916D
:102E2000F202992319F091509093F202882351F005
:102E30006091EE027091EF028091F0029091F102A8
:102E40000C94CF16089581E00C940F1770E00C9449
:102E5000401D609110018091EE0280FF0AC08091B8
:102E60000F0123E0829FC00111248D509D4F0C94CF
:102E700026178091110190911201891780F7E82F90
:102E8000F0E09F01220F331FE20FF31FED50FD4FC3
:102E90001182108212828F5FF0CF9091EE0290FF2C
:102EA00016C09091110120911201921770F4E92F30
:102EB000F0E0DF01AA0FBB1FEA0FFB1FED50FD4F33
:102EC0008183608342839F5FF0CF0C94291708951C
:102ED000CF93DF9300D01F92CDB7DEB79091EE0273
:102EE00090FF0AC09E012F5F3F4F0E94AA164B81A0
:102EF00069818A810E944D170F900F900F90DF918A
:102F0000CF910895CF93DF93EC01EC81F0E0E65F81
:102F1000FD4F4491EEEEF2E0628181810E946817DC
:102F20008C818F5F8C83DF91CF910895CF93DF9356
:102F3000EC01EEEEF2E0438162818C810E94681721
:102F40008C818F5F8C83DF91CF9108950F931F93B6
:102F5000CF93DF9300D01F92CDB7DEB78C01809165
:102F60009B0281110AC09E012F5F3F4F4FEF6FEF11
:102F70000E94AA168A8180939B02F8018481813085
:102F800051F028F0823061F440919B020AC0809198
:102F90009B0240E007C060919B0240E080E003C0DC
:102FA00040E080E060E00E944D17F801848190E0ED
:102FB000019663E070E00E94D22884830F900F9006
:102FC0000F90DF91CF911F910F910895AF92BF9213
:102FD000CF92DF92EF92FF920F931F93CF93DF93E5
:102FE00000D01F92CDB7DEB7182FF62E042FE22E99
:102FF0009091EE0290FF6DC0E92FE695AE2FB0E004
:10300000A156BE4F8C918093A7029E7F923061F4AF
:103010009E012F5F3F4F812F0E94AA164B8169812D
:103020008A810E944D1743C0823019F40091F10249
:103030003EC0863019F41091EF0239C08930D9F3BF
:103040008931A9F5E9518E2F8170D82EE695F0E0EF
:10305000E65FFC4FA590B490C12CBB246091130196
:10306000C61618F52C2D30E0A29EC001A39E900D2F
:10307000B29E900D112470E00E94BE28812FD110C5
:1030800002C0860F01C0861B90911101290F311DCE
:10309000A901440F551F240F351F2D503D4F402FC0
:1030A0006F2D0E94AA16C394D9CF0E94291710939E
:1030B000EF02F092F0020093F102EE2051F06091E5
:1030C000EE027091EF028091F0029091F1020E9465
:1030D000CF160F900F900F90DF91CF911F910F910E
:1030E000FF90EF90DF90CF90BF90AF900895EEEEFD
:1030F000F2E09181282F438162818AE0890F0C944C
:10310000E61781E00C947718EEEEF2E09181282F1B
:103110004381628186EF890F0C94E61781E00C945D
:103120008418EEEEF2E062812AE0620F08F46FEF9D
:10313000282F438181810C94E61781E00C9491182B
:10314000EEEEF2E062812AE0621B08F460E0282FD4
:10315000438181810C94E61781E00C94A018EEEE77
:10316000F2E043812AE0420F08F44FEF282F6281FA
:1031700081810C94E61781E00C94AF18EEEEF2E03A
:1031800043812AE0421B08F440E0282F62818181BC
:103190000C94E61781E00C94BE1820E00C94E6171E
:1031A000FF920F931F93CF93DF93EC01F12C0FEF5E
:1031B00010E060911301F616F0F4809111012F2DAB
:1031C00030E0280F311DC901880F991F280F391FC2
:1031D0002D503D4F70E0C8010E94D228962F8C815F
:1031E0004091F1026091F002F99E800D11240E943D
:1031F000AA16F394DECF0E9429179A818C8190FF42
:1032000002C08F5F01C081508C83DF91CF911F91ED
:103210000F91FF900895BF92CF92DF92EF92FF92AD
:103220000F931F93CF93DF93FC01828180FF02C035
:103230000FEF01C001E010E080911301181708F0B2
:1032400040C080911101C12ED12CE601C80FD11DC3
:10325000CE01880F991FC80FD91FCD50DD4F19829D
:1032600018821A8234E0E32EF12CB12C80919D0259
:103270008B0D813114F08F7005C087FF03C09091D2
:103280001301890F082E000C990BC816D90691F46A
:103290008091F1028E9DA0018F9D500D11245595B6
:1032A0004795559547959E016091F0028091EF02F8
:1032B0000E94AA16B00EF1E0EF1AF108B9F61F5FEE
:1032C000BBCF0E94291780919D02013031F48111FA
:1032D00002C080911301815007C090E00196609177
:1032E000130170E00E94D22880939D02DF91CF915C
:1032F0001F910F91FF90EF90DF90CF90BF900895B6
:10330000CF938091110190911201891770F4E82FE9
:10331000F0E09F01220F331FE20FF31FED50FD4F2E
:103320001182108212828F5FF0CFC0E06091130192
:10333000C617C0F5EC2FF0E070E0CF010E94D22854
:1033400020911101820F20919C02022E000C330B60
:1033500090E0E217F307CCF020910E01022E000C52
:10336000330B2E173F078CF09C01220F331F820F67
:10337000931F9C012D503D4F4091F1026091F0024E
:103380008091EF020E94AA160BC0FC01EE0FFF1FF6
:103390008E0F9F1FFC01ED50FD4F11821082128293
:1033A000CF5FC4CF0E94291720910D0180919C020C
:1033B000820F80939C0290910E01920F90930E01C8
:1033C00019165CF4082E000C990B4091130150E083
:1033D00041505109841795071CF0219520930D0148
:1033E000CF9108958F929F92AF92BF92CF92DF922A
:1033F000EF92FF920F931F93CF93DF938C01FC0109
:103400004481C42FD0E09E01DE010E9416299B0159
:10341000AC010E942C296B017C01E0E2F0E0EC1B86
:10342000FD0BA5E5B0E09B01AC010E942C294B01EE
:103430005C019F01DF010E940E299B01AC010E94EB
:1034400037299B01AC012C0D3D1D4E1D5F1DC50193
:10345000B4010E94E628C22FD22F2A3228F4F3E0CA
:103460002F9F900111240DC025E530E02C1B310960
:10347000C901880F991F280F391F37FF02C02F5F1E
:103480003F4F35952795C22FC095F12C85E5E82E45
:10349000ED1A80911301F816C8F4F1FC02C08E2DCC
:1034A00001C08D2F909111012F2D30E0290F311D7A
:1034B000A901440F551F240F351F2D503D4F4C2F90
:1034C0006091F0020E94AA16F394E3CF0E9429179C
:1034D000F8018481811102C091E003C0803219F4A7
:1034E0009FEF90930C0190910C01890FF801848358
:1034F000DF91CF911F910F91FF90EF90DF90CF90D0
:10350000BF90AF909F908F9008950F931F93CF938C
:10351000DF93EC0100E010E080911301282F30E0F0
:103520000217130724F5909111019801290F311DFD
:10353000A901440F551F240F351F2D503D4F86956F
:1035400090E04C81081719071CF4442331F002C0A5
:10355000411103C04091F10201C040E06091F002CE
:103560008091EF020E94AA160F5F1F4FD5CF0E94D5
:1035700029178C8190E00196817099278C83DF91C7
:10358000CF911F910F910895EEEEF2E080818E7F32
:10359000808360817181828193810E94CF16109215
:1035A000A8022FEF80E792E0215080409040E1F7A1
:1035B00000C000000C942917EEEEF2E080818E7FAF
:1035C00080831092A8022FEF80E792E02150804084
:1035D0009040E1F700C000000C9429171092A80257
:1035E0008091A50281110AC081E08093A50280919B
:1035F000EE0281708093A4020C94DC1A089560910D
:10360000EE02669570E04BE050E084E191E00E94AC
:103610003F29892B19F481E08093A8020E946C2134
:1036200090939F0280939E0208959091EE0290FFE6
:1036300035C09170811102C0926006C0853210F0D1
:10364000986402C0880F982B9093EE02662351F085
:103650006091EE027091EF028091F0029091F10280
:103660000E94CF166091EE02669570E04BE050E04C
:1036700084E191E00E943F29892B19F01092A80261
:1036800002C00E94FF1A81E08093A1024091F102E2
:103690006091F0028091EF020C94CD180895682F8C
:1036A0009091EE02969581E0890F853208F081E0D5
:1036B0000C94151B81E00C944F1B682F9091EE0227
:1036C00096958FEF890F09F484E20C94151B81E025
:1036D0000C945D1B61E00C94151BEEEEF2E0808112
:1036E0008160808386950C946A1B8091EE0280FD38
:1036F0000C94C41A0C946D1B60E00C94151B809103
:10370000A60281112EC00E94610E811104C00E9488
:10371000090F0E94E1160E94CB166093EE0270938F
:10372000EF028093F0029093F1026E7F61F40E94A9
:10373000E1160E94CB166093EE027093EF02809325
:10374000F0029093F1020E94B8161092A8028091A4
:10375000EE0280FF03C086950E947C1B81E080936F
:10376000A6020895EEEEF2E0808181608083869566
:103770000C947C1B1092A5028091A40281110E94DE
:10378000B21B0C94FF1A0F931F93CF93DF9380917A
:10379000A802882309F485C08091A702E091EE0277
:1037A000E695E81BE093A002823049F4F0E0EA5F7E
:1037B000FD4FE491CE2FD0E002E817E149C08630FA
:1037C00049F4F0E0ED5FFD4FE491CE2FD0E006E943
:1037D00017E13EC0893051F4E695F0E0E050FE4F2D
:1037E000E491CE2FD0E000ED18E132C08F3051F4DB
:1037F000E695F0E0E350FE4FE491CE2FD0E00BE0F1
:1038000019E126C0853149F4F0E0E650FE4FE4911D
:10381000CE2FD0E000E819E11BC0883181F083325F
:1038200039F4E8EFF1E0C591D49106EA17E110C050
:10383000843251F4C4EFD1E005E81AE109C0C8E2CE
:10384000D0E002EF19E104C0C0EDD7E006EA16E1CE
:103850008091A102882361F01092A1020E946C2144
:1038600090939F0280939E021092A3021092A20254
:103870000E946C21E0919E02F0919F028E1B9F0B93
:103880008F3F9F4770F4EC0FFD1FF0939F02E09372
:103890009E028EE992E0F801DF91CF911F910F9186
:1038A0000994DF91CF911F910F910895882311F012
:1038B000FA0101C0FB010994CF93DF93C82FD62FE3
:1038C0000E94F0168C1740F00E94F0168D1720F41D
:1038D000DF91CF910C945A1B8C2FDF91CF910C94D8
:1038E0006A1B1F93CF93DF93FB0112811111C3C099
:1038F000EC010E94780D8272CD3CFCE5DF0709F4F3
:103900009AC0A8F5C73CECE5DE0709F476C0A8F438
:10391000C43C9CE5D90709F45FC028F4C33CDC45EE
:1039200009F457C054C0C53C9CE5D90709F459C0F7
:10393000C63CDC4509F45CC04AC0CA3CFCE5DF0774
:1039400009F46AC050F4C83CECE5DE0709F45AC03B
:10395000C93CDC4509F45BC03AC0CB3C9CE5D907C7
:1039600009F45FC0CC3CDC4509F460C030C0C23D06
:10397000FCE5DF0709F46FC088F4CF3C9CE5D9076C
:1039800009F460C008F45CC0C03DFCE5DF0709F441
:103990005CC0C13DDC4509F45BC019C0C53D9CE578
:1039A000D90709F460C050F4C33DFCE5DF0709F412
:1039B00055C0C43DDC4509F454C009C0C63D9CE572
:1039C000D90709F455C0CE35DD4509F454C011E0DE
:1039D00052C00E94751B4FC047E65BE16AE57BE180
:1039E00004C04AE55BE167E67BE10E94561C43C0E8
:1039F0004EE858E161E878E1F8CF41E858E16EE837
:103A000078E1F3CF4CEA58E16DE978E1EECF4DE98A
:103A100058E16CEA78E1E9CF4AEC58E16BEB78E1E8
:103A2000E4CF4BEB58E16AEC78E1DFCF43E257E1BA
:103A30006CE077E1DACF4CE057E163E277E1D5CF94
:103A400081E017C065E082E010C068E086E00DC04C
:103A50006EE089E00AC064E18FE007C067E185E1BC
:103A600004C088E106C062E289E10E945C1C03C0D8
:103A700083E20E946A1B812FDF91CF911F910895ED
:103A80003F9A28B12F7738B130684FB7F894FC01CE
:103A9000CB01880F991F680F791F6E0F7F1FE617E4
:103AA000F70789F0819198E038B9000000C087FFDE
:103AB00028B9880F000000C000C000C028B900C0AD
:103AC0009A9591F7ECCF4FBF8FE594E00197F1F70E
:103AD00000C000000895CF93DF93EC01FB018281C9
:103AE000882309F43CC1C430FDE5DF0760F4CB3F17
:103AF0009CE5D90788F49E0122503C4524313105CC
:103B000008F02EC109C0C236EDE5DE0729F0C63A3D
:103B1000FDE5DF0709F024C10E94740E9093DB02DB
:103B20008093DA02C1318CE5D80709F4C6C008F0E9
:103B300042C0C930ECE5DE0709F49BC000F5C53092
:103B40008CE5D80709F485C078F4C330ECE5DE07CE
:103B500009F478C008F07AC0C230DC4509F0F5C03D
:103B60008091DA028160EFC0C7309CE5D90709F483
:103B700078C008F07AC08091DA028061E4C0CD306C
:103B8000FCE5DF0709F487C058F4CB309CE5D90782
:103B900009F479C008F07BC08091DA0288606FC0B8
:103BA000CF30FCE5DF0709F480C008F082C08091C7
:103BB000DA02877FC8C0CE3F9CE5D90709F471C0FF
:103BC00000F5C531FCE5DF0709F485C068F4C331B1
:103BD0009CE5D90709F475C008F095C00E94250836
:103BE0008091DA028F77AFC0CC3FFCE5DF07A9F107
:103BF00008F054C0CB3FDC4509F0A7C08091DB0240
:103C000040C0C230EDE5DE0709F489C058F4C115A3
:103C10008DE5D80709F45AC008F069C08091DB022D
:103C200082602FC0C236EDE5DE0709F47CC0C63ADB
:103C3000FDE5DF0709F481C0C330DD4509F085C02B
:103C400080E06EC08091DA0282607DC08091DA02ED
:103C500016C08091DA02886076C08091DB028260B3
:103C60004FC08091DA0280626EC08091DA02806477
:103C70006AC00E9425088091DA02806864C084606E
:103C800062C081603DC08091DA028E7F5CC080910D
:103C9000DA028D7F58C08091DA0216C08091DB0273
:103CA00018C08091DB028D7F2BC08091DA028F7E5D
:103CB0004AC08091DA028F7D46C08091DA028F7B04
:103CC00042C08091DA02877F8B7F3DC08091DB020A
:103CD0008D7F8E7F15C08091DA0282FB222720F92A
:103CE00091E0922790FB82F990FB83F92CC08091A0
:103CF000DB02982F909591708E7F892B90FB81F934
:103D00008093DB0222C00E9425088091DA0287FBA3
:103D1000222720F991E0922790FB87F914C081E0D7
:103D20000E940B0F12C08091DA0284FB222720F937
:103D300091E0922790FB84F906C08091DA02982FD7
:103D4000909590FB80F98093DA028091DA0290914D
:103D5000DB020E94850E0E94250880E001C081E000
:103D6000DF91CF910895CF93DF9386319C4541F544
:103D7000EB010E94780D982F8A81209102013091E9
:103D80000301882379F09A7A81E009F480E0809336
:103D9000A902911102C069E201C065E3C9010E9454
:103DA000A9200AC08091A902811102C069E201C064
:103DB00065E3C9010E94B4200E94BA0D80E001C0F1
:103DC00081E0DF91CF9108950F931F93CF93DF93FD
:103DD000C42FD22FFC0182818823C9F04093AC020A
:103DE0000E946C219093AB028093AA0280E28C0F18
:103DF000883008F057C0C77081E001C0880FCA95AD
:103E0000EAF7DF91CF911F910F910C948205809179
:103E1000AC02481330C08091AA029091AB020E947C
:103E20008421883C910538F510E21D0FCD17B9F0BB
:103E300080E28C0F883040F4C77081E001C0880FA9
:103E4000CA95EAF70E948905183028F581E09D2F70
:103E5000977001C0880F9A95EAF70E948205802F1B
:103E60000E9479051830F0F4D77081E001C0880F06
:103E7000DA95EAF70AC080E28C0F883098F4C770B0
:103E800081E001C0880FCA95EAF7DF91CF911F91B9
:103E90000F910C948905802FDF91CF911F910F9185
:103EA0000C947905DF91CF911F910F9108950F9395
:103EB0009C01CB01243F4CE5340731F188F4293DC6
:103EC000FCE53F07D9F02A3D4CE5340779F1283D60
:103ED0003C45A9F506E221EE41EE68ED7CE52BC0FC
:103EE000263FFCE53F07E1F0A8F0273F3C4539F5C8
:103EF00007E225EE46EE67EF7CE51DC007E225EE02
:103F000045EE69ED7CE517C006E221EE40EE64EF78
:103F10007CE511C007E225EE44EE65EF7CE50BC0C1
:103F200006E221EE42EE66EF7CE505C008E221E004
:103F300045EE6AED7CE50E94E41E80E008C0FC01CD
:103F40008281882319F01092AC0201C081E00F91A8
:103F500008959093C5018093C40108959093B2028F
:103F60008093B1020895E091B102F091B2023097CE
:103F700021F00190F081E02D099480E00895E09116
:103F8000B102F091B202309799F020912B012223D7
:103F900059F02091DA0227FF07C0DC012C9111961D
:103FA0002C93119726E02C930280F381E02D099445
:103FB0000895E091B102F091B202309739F022E019
:103FC000DC012C930480F581E02D09940895209163
:103FD000AF023091B0022817390771F09093B00208
:103FE0008093AF02E091B102F091B202309721F0DC
:103FF0000680F781E02D099408952091AD0230915B
:10400000AE022817390771F09093AE028093AD028B
:10401000E091B102F091B202309721F00084F18575
:10402000E02D09940895FC01329680912B0188239C
:1040300031F08091DA0287FF02C09EE101C096E074
:1040400080E0915028F021912223D9F38F5FF9CF9E
:104050000895662351F120912B012223E9F020914C
:10406000DA0227FF19C0462F4695469546954E31F0
:10407000E0F4677021E030E002C0220F331F6A9540
:10408000E2F7FC01E40FF11D828190E0282339233F
:1040900081E0232B69F409C0FC0132960896219136
:1040A000621729F0E817F907D1F780E0089581E059
:1040B00008959C01FC0132969FEF80E041914617E4
:1040C00089F09F3F19F4411101C0982F8F5F86300E
:1040D000A9F79F3F39F0F901E90FF11D97FDFA9516
:1040E0006283089508959C012A5F3F4FFC0142813D
:1040F000461301C01282019682179307B9F70895FB
:10410000262F2695269526952E3168F4FC01E20F80
:10411000F11D677021E030E001C0220F6A95EAF7D7
:104120008281282B22830895262F26952695269571
:104130002E3170F4FC01E20FF11D677021E030E0D8
:1041400001C0220F6A95EAF72095828128232283F5
:10415000089520912B01222329F02091DA0227FDD6
:104160000C9480200C94592020912B01222329F0BB
:104170002091DA0227FD0C9494200C947320209156
:104180002B01FC013296222331F08091DA0287FF65
:1041900002C08EE101C086E0DF011D928A95E9F739
:1041A000089508950C94D12083E08093B3020C9479
:1041B000D220811102C081E001C082E08093B3026D
:1041C0000C94D2200C94D92081E08093B3020C94FB
:1041D000D2200C94E42008950C94EB200C94EC2055
:1041E0000C94EB200C94EB200C94EB20CF930E94CA
:1041F000F2200E94EE120E94F020C0E08C2F0E945C
:104200002612811104C0CF5FC930C1F701C081E01F
:10421000CF91089508951F920F920FB60F92112417
:104220008F939F93AF93BF938091B402811113C07A
:104230008091230390912403A0912503B09126033C
:104240004196A11DB11D8093230390932403A09355
:104250002503B0932603BF91AF919F918F910F904B
:104260000FBE0F901F90189580912B03843031F171
:104270000E94D1031092B40220E488E190E00FB6CE
:10428000F894A895809360000FBE2093600083B7D8
:10429000817F846083BF83B7816083BF7894889572
:1042A00083B78E7F83BF0FB6F894A8958091600086
:1042B000886180936000109260000FBE08950E9494
:1042C00025080C94D70382E084BD93E095BD9AEF56
:1042D00097BD80936E0008952FB7F89480912303C3
:1042E00090912403A0912503B09126032FBF089538
:1042F0002FB7F894609123037091240380912503D4
:10430000909126032FBF08959C014FB7F894809198
:10431000230390912403A0912503B09126034FBF5E
:10432000821B930B089578941F920F920FB60F92F1
:1043300011248F939F93AF93BF9380912303909108
:104340002403A0912503B09126030196A11DB11D60
:104350008093230390932403A0932503B093260313
:10436000BF91AF919F918F910F900FBE0F901F90B3
:10437000189581E08093E00080E28093D80010924D
:10438000C9008FE19EE40197F1F700C0000087E0CB
:1043900090EBDC018093340390933503A0933603B4
:1043A000B09337039CE088E10FB6F894A89580930A
:1043B00060000FBE90936000FFCF8091D8020895F7
:1043C000089522E02093E9002FEF3091E80021507A
:1043D00035FD06C035ED3A95F1F700002111F5CF16
:1043E0002091E80025FF0BC040E050E066E070E05F
:1043F0000E9420248091E8008E778093E800089541
:10440000CF93DF9320912B01222339F02091DA0200
:1044100027FF03C060E222E002C068E021E02093B1
:10442000E9002FEF3091E800215035FD06C035ED51
:104430003A95F1F700002111F5CF2091E80025FF12
:104440001DC0EC0180912B01811105C040E050E0BE
:1044500068E070E003C070E040E050E0CE010E94F0
:1044600020248091E8008E778093E80080E2FE01AE
:10447000A8EBB2E001900D928A95E1F7DF91CF9120
:1044800008958093B5027093B7026093B60280914D
:104490002B03843001F582E08093E9008FEF909147
:1044A000E800815095FD06C095ED9A95F1F7000062
:1044B0008111F5CF8091E80085FF0DC040E050E00C
:1044C00063E070E085EB92E00E9420248091E80098
:1044D0008E778093E8000895BC0184E00C9441221B
:1044E000BC0183E00C94412280912A03811109C010
:1044F0000E94B1250E940E268091E2008460809384
:10450000E200089510922A0308950C94E920609126
:10451000270381E0611101C080E00C94D4209091C8
:104520002B0381E0943009F080E0609127030C9424
:10453000D92042E061EC81E00E942A2542E261EC50
:1045400082E00E942A2590912B0381E0943009F0AB
:1045500080E0609127030C94E22080912D0383304A
:1045600009F461C030F4813071F0823009F49AC0EE
:1045700008958A3009F486C08B3009F46CC0893004
:1045800009F0A8C020C080912C03813A09F0A2C094
:104590008091E800877F8093E800809130039091BC
:1045A0003103892B21F460E288EB92E003C060E0E4
:1045B00080E090E070E00E946B248091E8008B77AF
:1045C0008093E800089580912C03813209F082C025
:1045D0008091300390913103029708F07BC0809165
:1045E000E800877F8093E8008091E80082FD05C0A5
:1045F00080912B038111F8CF6DC02091F300809141
:10460000F20090E0922B029731F48091F10081301A
:1046100011F0863021F48091F1008093D8028091CE
:10462000E8008B7753C080912C03813A09F052C087
:104630008091300390913103892B09F04BC0809118
:10464000E800877F8093E8008091E80080FFFCCF3E
:1046500080912B0136C080912C038132D9F5809155
:10466000300390913103892BA9F58091E800877F71
:104670008093E8000E945F2580912E0380932B0198
:104680000C94250880912C03813221F58091E8005B
:10469000877F8093E8000E945F2580912F0380939D
:1046A000D902089580912C03813AA1F48091E80009
:1046B000877F8093E8008091E80080FFFCCF8091A5
:1046C000D9028093F1008091E8008E778093E80012
:1046D0000C945F25089584B7877F84BF0FB6F89444
:1046E000A8958091600088618093600010926000BE
:1046F0000FBE90E080E80FB6F8948093610090932D
:1047000061000FBE0C94E4200E94B1250E940E2689
:10471000E2EEF0E080818460808378940C94A3289A
:104720008FE191E00C94AE1F80912B038530A9F4AA
:1047300080912B03853079F40E94342180912903E4
:104740008823B1F30E94F620882391F30E940A2463
:104750000E942508EDCF0C945F21089508950C94D4
:10476000B123292F332723303105C9F060F42130DC
:10477000310581F02230310509F044C08BE390E02F
:1047800023E434E043C021323105E1F02232310527
:1047900049F138C082E190E02EE734E037C0992734
:1047A0008130910549F028F0029761F5EFE0F4E0DF
:1047B00005C0EFE3F4E002C0EFE2F4E0849190E0A2
:1047C0009F0124C06115710541F061307105D1F47C
:1047D00089E090E02EE634E019C089E090E025E51C
:1047E00034E014C06115710541F06130710551F478
:1047F00086EB90E020E934E009C080E490E026E414
:1048000035E004C080E090E020E030E0FA01318340
:104810002083089580E189BD82E189BD09B400FE4D
:10482000FDCF8091D8008F7D8093D8008091E000EB
:1048300082608093E0008091E00081FDFCCF0895CC
:10484000CF92DF92EF92FF920F931F93CF93DF935C
:10485000EC018B017A010E947E25811133C0E114A5
:10486000F10439F0F70180819181081B190BC80F01
:10487000D91FC12CD12C0115110519F18091E80027
:1048800085FD16C08091E8008E778093E800E114E2
:10489000F10449F0F70180819181C80ED91ED182BF
:1048A000C08285E00FC00E947E25882321F30AC0C4
:1048B00089918093F10001501109FFEFCF1ADF0AAF
:1048C000DACF80E0DF91CF911F910F91FF90EF90B1
:1048D000DF90CF9008952091320330913303261753
:1048E000370748F06115710539F42091E8002E77FB
:1048F0002093E80001C0B901FC0120E061157105B9
:1049000079F180912B038823F1F18530F1F18091C9
:10491000E80083FD3CC08091E80082FD2EC08091BC
:10492000E80080FFEBCF2091F3008091F20090E04F
:10493000922B6115710551F08830910538F4219161
:104940002093F100615071090196F3CF21E008979F
:1049500009F020E08091E8008E778093E800CECFC8
:104960002111CFCF0AC080912B03882361F08530BD
:1049700061F08091E80083FD0AC08091E80082FF29
:10498000F2CF80E0089582E0089583E0089581E009
:10499000089520913203309133032617370748F0EA
:1049A0006115710539F42091E8002E772093E80015
:1049B00001C0B901FC0120E06115710591F1809100
:1049C0002B03882309F440C0853009F43FC080914F
:1049D000E80083FD3DC08091E80082FD2FC08091FA
:1049E000E80080FFE9CF2091F3008091F20090E091
:1049F000922B6115710559F08830910540F424918E
:104A00002093F1003196615071090196F2CF21E0B7
:104A1000089709F020E08091E8008E778093E80005
:104A2000CBCF2111CCCF0AC080912B03882361F01A
:104A3000853061F08091E80083FD0AC08091E80034
:104A400082FFF2CF80E0089582E0089583E0089528
:104A500081E00895982F973068F59093E9009817B2
:104A600039F07091EC002091ED005091F00003C0FE
:104A7000242F762F50E021FD02C09F5FECCF3091B4
:104A8000EB003E7F3093EB003091ED003D7F3093A3
:104A9000ED003091EB0031603093EB007093EC004F
:104AA0002093ED005093F0002091EE0027FDE5CF1C
:104AB00080E008958F708093E90081E008958091EF
:104AC0002C0387FF11C08091E80082FD05C0809112
:104AD0002B038111F8CF11C08091E8008B770BC0B8
:104AE00080912B03882349F08091E80080FFF8CF64
:104AF0008091E8008E778093E80008952091E4008B
:104B00003091E50095E64091EC00842F817040FFE4
:104B100023C08091E80080FD1DC080912B03882375
:104B200099F0853099F08091EB0085FD11C040919E
:104B3000E4005091E5002417350729F3915011F056
:104B40009A01E1CF84E0089582E0089583E008951A
:104B500081E0089580E008954091E80042FFDDCFB4
:104B600008950E941F260E942726E0EEF0E0808133
:104B700081608083E8EDF0E080818F77808319BCCD
:104B8000A7EDB0E08C918E7F8C9380818F7E8083A7
:104B900010922A0308950F931F93CF93DF930E94DF
:104BA0001F260E942726C8EDD0E088818F77888352
:104BB00088818068888388818F7D888319BC109262
:104BC0002B0310922703109229031092280300EE62
:104BD00010E0F80180818B7F8083888181608883E9
:104BE00042E060E080E00E942A25E1EEF0E0808172
:104BF0008E7F8083E2EEF0E080818160808380811F
:104C000088608083F80180818E7F808388818061C5
:104C10008883DF91CF911F910F910895E8EDF0E027
:104C200080818F7E8083E7EDF0E0808181608083EA
:104C300084E082BF81E080932A030C94CB25E8EDC9
:104C4000F0E080818E7F80831092E20008951092C0
:104C5000DA001092E10008951F920F920FB60F92A2
:104C600011242F933F934F935F936F937F938F9371
:104C70009F93AF93BF93EF93FF938091E10082FFE7
:104C80000BC08091E20082FF07C08091E1008B7F22
:104C90008093E1000E94A2288091DA0080FF1FC06B
:104CA0008091D80080FF1BC08091DA008E7F8093B6
:104CB000DA008091D90080FF0DC080E189BD82E1DA
:104CC00089BD09B400FEFDCF81E080932B030E94D3
:104CD000742205C019BC10922B030E94822280917D
:104CE000E10080FF19C08091E20080FF15C0809133
:104CF000E2008E7F8093E2008091E20080618093E9
:104D0000E2008091D80080628093D80019BC85E0D1
:104D100080932B030E9487228091E10084FF30C0A2
:104D20008091E20084FF2CC080E189BD82E189BDD1
:104D300009B400FEFDCF8091D8008F7D8093D8000C
:104D40008091E1008F7E8093E1008091E2008F7E70
:104D50008093E2008091E20081608093E200809184
:104D60002703882311F084E007C08091E30087FDCA
:104D700002C081E001C083E080932B030E948F2258
:104D80008091E10083FF29C08091E20083FF25C06C
:104D90008091E100877F8093E10082E080932B0384
:104DA000109227038091E1008E7F8093E100809133
:104DB000E2008E7F8093E2008091E2008061809328
:104DC000E20042E060E080E00E942A258091F0004D
:104DD00088608093F0000E948522FF91EF91BF913F
:104DE000AF919F918F917F916F915F914F913F9183
:104DF0002F910F900FBE0F901F9018951F920F923A
:104E00000FB60F9211242F933F934F935F936F939D
:104E10007F938F939F93AF93BF93CF93DF93EF9342
:104E2000FF93C091E900CF708091EC00D82FD17032
:104E300080FDD0E81092E9008091F000877F809398
:104E4000F00078940E9442271092E9008091F000CF
:104E500088608093F000CD2BCF70C093E900FF9164
:104E6000EF91DF91CF91BF91AF919F918F917F9102
:104E70006F915F914F913F912F910F900FBE0F90C7
:104E80001F9018951F93CF93DF93CDB7DEB7AA97E6
:104E90000FB6F894DEBF0FBECDBFECE2F3E0809119
:104EA000F100819323E0E433F207C9F70E94AD22B9
:104EB0008091E80083FF2EC180912C0390912D03F7
:104EC000492F50E04A30510508F024C1FA01EE594B
:104ED000FF4F0C940829803821F0823809F01AC15C
:104EE00008C08091280390912903992389F082605A
:104EF0000FC0809130038F70873008F00BC1809312
:104F0000E9008091EB0085FB882780F91092E90089
:104F10009091E800977F9093E8008093F1001092C1
:104F2000F100D1C0282F2D7F09F0F4C0882319F09B
:104F3000823061F0EFC080912E03813009F0EAC029
:104F4000933009F080E0809329032EC080912E03D6
:104F500081112AC0809130038F702FEF280F2630E7
:104F600008F0D8C08093E9002091EB0020FF1CC01E
:104F7000933021F48091EB00806214C09091EB009B
:104F800090619093EB0021E030E0A90102C0440F52
:104F9000551F8A95E2F74093EA001092EA0080914B
:104FA000EB0088608093EB001092E9008091E800AC
:104FB000877F8093E8000E945F25ACC08111AAC062
:104FC00010912E031F778091E3008078812B8093CE
:104FD000E3008091E800877F8093E8000E945F25CE
:104FE0008091E80080FFFCCF8091E300806880938F
:104FF000E300111102C082E001C083E080932B0323
:1050000089C08058823008F085C080912E0390912D
:105010002F038C3D53E0950779F583E08A838AE27C
:1050200089834FB7F894DE01139620E03EE051E209
:10503000E32FF0E050935700E49120FF03C0E29586
:10504000EF703F5FEF708E2F90E0EA3010F0C79660
:1050500001C0C0968D939D932F5F243149F74FBFB8
:105060008091E800877F8093E8006AE270E0CE01DB
:1050700001960E946B2416C0609130037091310339
:10508000AE014F5F5F4F0E94AF23BC01892B09F433
:1050900041C09091E800977F9093E80089819A81C0
:1050A0000E94C9248091E8008B778093E80032C089
:1050B000803881F58091E800877F8093E8008091B7
:1050C00027038093F1008091E8008E7772CF8111E1
:1050D00021C080912E0390912F0399270297D4F439
:1050E0008091E800877F8093E80080912E03809371
:1050F00027030E945F2580912703811106C08091BC
:10510000E30087FD02C081E001C084E080932B03AF
:105110000E9499228091E80083FF0AC08091E800F4
:10512000877F8093E8008091EB0080628093EB00A2
:10513000AA960FB6F894DEBF0FBECDBFDF91CF9118
:105140001F9108950895CF9380912B038823A1F098
:10515000C091E900CF709091EC00892F817090FD93
:1051600080E8C82B1092E9008091E80083FD0E943E
:105170004227CF70C093E900CF910895AA1BBB1BB3
:1051800051E107C0AA1FBB1FA617B70710F0A61B47
:10519000B70B881F991F5A95A9F780959095BC0168
:1051A000CD01089597FB072E16F4009407D077FDE4
:1051B00009D00E94BE2807FC05D03EF49095819549
:1051C0009F4F0895709561957F4F0895A1E21A2E23
:1051D000AA1BBB1BFD010DC0AA1FBB1FEE1FFF1F9B
:1051E000A217B307E407F50720F0A21BB30BE40BEB
:1051F000F50B661F771F881F991F1A9469F7609532
:105200007095809590959B01AC01BD01CF010895EB
:10521000EE0FFF1F0590F491E02D09940E941629CE
:10522000332312F48A1B9B0B0C942729A29FB001F5
:10523000B39FC001A39F700D811D1124911DB29FCA
:10524000700D811D1124911D08950E941629B7FF2C
:105250000895821B930B08950E941629A59F900D17
:10526000B49F900DA49F800D911D11240895B7FF48
:105270000C942C290E942C29821B930B0895FC016D
:105280004150504030F001900616D1F73197CF01D0
:105290000895882799270895FB01DC0104C08D91AA
:1052A0000190801921F441505040C8F7881B990B98
:1052B0000895F999FECF92BD81BDF89A992780B5DE
:1052C0000895A6E1B0E044E050E00C949329A8E1F1
:1052D000B0E042E050E00C949329262FF999FECFDC
:1052E00092BD81BDF89A019700B4021639F01FBA39
:1052F00020BD0FB6F894FA9AF99A0FBE0895039656
:10530000272F0E946E290E946D29252F0E946E2949
:10531000242F0C946E290196272F0E946E290C943D
:105320006D29DC01CB01FC01F999FECF06C0F2BD6D
:10533000E1BDF89A319600B40D9241505040B8F753
:065340000895F894FFCF70
:10534600C8005702280850011E0A14010101020074
:105356001000101001191A1B1C1D1E1F202122DD12
:10536600210022E12170226C22E02101E200E90005
:10537600EA00B500B600B700CD008301CC008A0173
:105386009201940121022302240225022602270209
:105396002A02B300B4006F007000818283E200E944
:1053A60000EA00B500B600B700CD008301CC008A44
:1053B60001920194012102230224022502260227DA
:1053C600022A02B300B4006F0070008182839091BC
:1053D60092F7F6F5F4F16636343596979593940080
:1053E60001020202020606060909090909090F0F48
:1053F6000F0F0F0F1515151819191919191919194C
:045406001919232429
:00000001FF
